:10000000DAEF21F00000000000EF00F00000000037
:0A0010000000000000000000F3D71C
:08001C000AAE029E000E120064
:100024000B820BAE1CEF00F00368026801680068E5
:080034000A360232FF0E120031
:0E003C00026A016A006A086A036A000E120076
:10004A000B840BAE30EF00F0010E036E026A016AF8
:0A005A00006A0A360232FF0E12009F
:100064000CB074EF00F00CA21AEF01F00E6A000E4F
:1000740002648BEF00F0F00E0214D8A456EF00F0E7
:10008400023A01380F0B02260138F00B016E0038DA
:100094000F0B01260038F00B006E08380F0B0026FA
:1000A4000838F00B086E0E84D89002BE6FEF00F093
:1000B40008360036013602360E2A02BE6FEF00F013
:1000C40008360036013602360E2A02BE6FEF00F003
:1000D40008360036013602360E2A0E50036410EF3D
:1000E40001F0035E0BBC08AE15EF01F0D880800E62
:1000F40008640030000E002201220222D8A015EF6D
:1001040001F0023201320032034A1AEF01F015EF16
:1001140001F001C002F000C001F008C000F0086A5C
:10012400000E0E860264C2EF00F0F00E0214D8A492
:10013400AAEF00F0023A01380F0B02260138F00B47
:10014400016E00380F0B01260038F00B006E0E8490
:10015400D89002BE6FEF00F00036013602360E2A48
:1001640002BE6FEF00F00036013602360E2A02BEE0
:100174006FEF00F00036013602360E2A6FEF00F002
:1001840001C002F000C001F0006A000E0E960E8855
:100194000264EFEF00F0F00E0214D8A4DAEF00F0DE
:1001A400023A01380F0B02260138F00B016E0E845F
:1001B400D89002BE6FEF00F0013602360E2A02BE5E
:1001C4006FEF00F0013602360E2A02BE6FEF00F028
:1001D400013602360E2A6FEF00F001C002F0016A08
:1001E400000E0E8602641FEF01F0F00E0214D8A474
:1001F400FEEF00F0023A0E84D89002BE6FEF00F0DA
:1002040002360E2A02BE6FEF00F002360E2A02BE3C
:100214006FEF00F002360E2A6FEF00F0010E0C6E45
:1002240012DF22EF01F0020E0C6EF6DE22EF01F077
:10023400040E0C6EF5DE22EF01F0080E0C6EFCDEEF
:020244001200A6
:0E024600ACB202D00000FCD7A1C1ADFF120087
:10025400A1C16FFF6DB002D00000FCD76FCF00F0DA
:02026400120086
:0C02660072B201D0FDD7A1C173FF1200DD
:100272000D6A086A0050D8B4000C04180A6E0ABE4F
:100282000D1E0B6A04AE02D0041E042A00AE02D078
:10029200001E002A005004100A6E0ABE1FD004502D
:1002A200085E003600340836045008260036060E72
:1002B2000C6E00340836045000B0085E00A0082618
:1002C20000360C2EF6D700A008260BB015D00DAEC6
:1002D200000C001E002A081E082A000C04AE09D0D9
:1002E20000BE04D00050086E006AF1D7006A002AEE
:1002F200000C001E0B2AD3D7082A0450085CD8A48D
:0E030200E6D7086A002A00AEE2D7FF0C120010
:10031000086A096A000E076203640DEF02F00250DA
:1003200006180A6E075003267E0ED8A09EEF01F035
:10033000035ED8B011EF02F0A2EF01F0035ED8A087
:1003400015EF02F0028E068E02C00EF001C00BF017
:1003500000C00DF000500402F4CF0CF00150050273
:10036000F4CF00F0F3CF08F00402F3500C26F45061
:100370000822000E00220D500502F3500C26F45006
:100380000822000E002202500402F3500826F45006
:10039000002202500502016A000E0122F3500026DD
:1003A000F45001220D500602F3500826F4500022AA
:1003B000026A000E012202220B500602F3500026B0
:1003C000F4500122000E02220E500602F3500126C4
:1003D000F450022202BEF5EF01F008360036013675
:1003E00002360306D8B415EF02F008EF02F0D88009
:1003F000800E08640030000E002201220222D8A0E4
:1004000008EF02F0023201320032034A11EF02F02B
:100410000AAE029E000E17EF02F0010E0FDE17EF7C
:1004200002F0020EFFDD17EF02F0040E0EDE1200E6
:10043000086A080E0C6E003408360450085ED8B006
:0E04400002D00826D89000360C2EF5D71200F8
:10044E00025006180E6E086A096A0B6A035007649A
:10045E001AEF03F006500A6E068E028E03500B6ED4
:10046E000750036E000E0B646AEF02F00B50075E2E
:10047E00D8B40BEF03F0070E0764D9EF02F0075E56
:10048E0000C008F001C000F002C001F0026A074E81
:10049E000BEF03F00764AEEF02F0075E00C008F04A
:1004AE0001C000F0016A074E0BEF03F007648CEFFA
:1004BE0002F0075E00C008F0006A074E0BEF03F073
:1004CE00076473EF02F00AC002F005C001F004C029
:1004DE0000F0086A35EF04F0030E07647EEF02F0B9
:1004EE00075E08380F0B086E074E0BEF03F0D8901F
:1004FE000832074E0BEF03F0D8900832074E0BEF81
:10050E0003F0D89008320BEF03F0030E07649DEF53
:10051E0002F0075E08380F0B086E0038F00B082645
:10052E0000380F0B006E074E0BEF03F0D890003221
:10053E000832074E0BEF03F0D89000320832074E08
:10054E000BEF03F0D890003208320BEF03F0030EDE
:10055E000764C5EF02F0075E08380F0B086E00380F
:10056E00F00B082600380F0B006E0138F00B00263A
:10057E0001380F0B016E074E0BEF03F0D8900132CE
:10058E0000320832074E0BEF03F0D89001320032E2
:10059E000832074E0BEF03F0D890013200320832CA
:1005AE000BEF03F0030E0764F6EF02F0075E083858
:1005BE000F0B086E0038F00B082600380F0B006E7C
:1005CE000138F00B002601380F0B016E0238F00BCC
:1005DE00012602380F0B026E074E0BEF03F0D89078
:1005EE000232013200320832074E0BEF03F0D89080
:1005FE000232013200320832074E0BEF03F0D89070
:10060E000232013200320832096A000E0EAEFFEFDE
:10061E0003F0081E001E011E021E082A00220122DF
:10062E000222FFEF03F00750D8A420EF03F035EFBE
:10063E0004F0096A02C00AF0028E068E0750035CAF
:10064E00076ED8B4F2EF03F0070E0764C0EF03F0A5
:10065E00075E0450096E0550046E0650056E066A5C
:10066E00074EF2EF03F0070E076495EF03F0075EF7
:10067E000450096E0550046E056A074EF2EF03F042
:10068E00070E076473EF03F0075E0450096E046AE9
:10069E00074EF2EF03F0070E07645AEF03F00AC09D
:1006AE0002F035EF04F0030E076465EF03F0075E0A
:1006BE0009380F0B096E074EF2EF03F0D89009328E
:1006CE00074EF2EF03F0D8900932074EF2EF03F027
:1006DE00D8900932F2EF03F0030E076484EF03F0B3
:1006EE00075E09380F0B096E0438F00B0926043823
:1006FE000F0B046E074EF2EF03F0D890043209325E
:10070E00074EF2EF03F0D89004320932074EF2EFA3
:10071E0003F0D89004320932F2EF03F0030E0764AF
:10072E00ACEF03F0075E09380F0B096E0438F00BBF
:10073E00092604380F0B046E0538F00B0426053815
:10074E000F0B056E074EF2EF03F0D8900532043210
:10075E000932074EF2EF03F0D89005320432093217
:10076E00074EF2EF03F0D890053204320932F2EF61
:10077E0003F0030E0764DDEF03F0075E09380F0B7D
:10078E00096E0438F00B092604380F0B046E053879
:10079E00F00B042605380F0B056E0638F00B0526F8
:1007AE0006380F0B066E074EF2EF03F0D8900632A6
:1007BE00053204320932074EF2EF03F0D8900632BA
:1007CE00053204320932074EF2EF03F0D8900632AA
:1007DE00053204320932086A000E0EAEFFEF03F046
:1007EE00091E041E051E061E092A042205220622C3
:1007FE0009500826045000220550012206500222FC
:10080E000EBE16EF04F0D8A025EF04F0023201322E
:10081E0000320832033E25EF04F02FEF04F0D8B07B
:10082E002AEF04F0000E081E001E011E021E082AEA
:10083E000022012202220A7E2AEF04F0010E0C6E23
:10084E000ADC37EF04F0020E0C6E05DC37EF04F015
:10085E00040E0C6E12EC00F037EF04F0000E0C6E6E
:02086E00120076
:100870000B800BAE44EF04F0026A0AAEFF0E026E6C
:0C088000016E006E0A360232FF0E1200FC
:10088C00A1C1C9FFC7B002D00000FCD7C9CF00F08E
:02089C00120048
:08089E000B6A0B86FF0E12002D
:1008A6000134083609360450085E0550D8A0053CC8
:1008B600095E003601360F0E0C6E01340836093615
:1008C600045000A006D0085E0550D8A0053C095E7D
:1008D60005D008260550D8B0053C09260036013655
:1008E6000C2EEBD700B006D0045008260550D8B021
:0808F600053C09260000120078
:0A08FE0000000000000000001200DE
:100908001D0E0C6E910E0D6E0D2EFED70C2EFCD703
:020918001200CB
:0C091A00420E0D6E0D2EFED700001200E4
:100926000450000A08E10550000A05E1FF0E006EBA
:100936007F0E016E57D00D6A096A086A01500010D1
:10094600D8B4000C015005180A6E0ABE0D1E0B6ABB
:1009560005AE05D0041E051E042AD8B4052A01AE2C
:1009660005D0001E011E002AD8B4012A0150051028
:100976000A6E0ABE10D094DF0BB020D00DAE000C6C
:10098600001E011E002AD8B4012A081E091E082AC4
:10099600D8B4092A000C05AE0DD001BE07D001500F
:1009A600096E0050086E016A006AE8D7016A006A9B
:1009B600002A000C011E001E0B2ADDD7082AD8B417
:1009C600092A0450085CD8A4D9D70550095CD8A4D4
:1009D600D5D7096A086A002AD8B4012A01AECED74B
:0609E6000000FF0C1200EE
:1009EC000450000A12E10550000A0FE10650000AFB
:1009FC000CE10750000A09E1FF0E006EFF0E016EBC
:100A0C007F0E026EFF0E036EA7D0086A096A0750AC
:100A1C00D8B4A1EF05F00350D8B4A5EF05F00250FF
:100A2C0006180A6E028E068E0E6A02C008F001C00D
:100A3C000CF000C00DF004500D5E0550D8A0053C24
:100A4C000C5E0650D8A0063C085E086A0C6A0D6A5B
:100A5C00D8A038EF05F0D8900232013200320832BB
:100A6C00010E0E6E0750035ED8A045EF05F07E0E0A
:100A7C000E240326D8B0AAEF05F04BEF05F07E0E3E
:100A8C000E240326D8A0AFEF05F0180E0B6E0D3612
:100A9C000C3608360036013602360E360450005E2F
:100AAC000550D8A0053C015E0650D8A0063C025E5D
:100ABC0006340E120EA066EF05F00D8071EF05F0F6
:100ACC00045000260550D8B0053C01260650D8B07D
:100ADC00062802260D900B2E4DEF05F097EF05F032
:100AEC00D8900036013602360E360450005E0550A2
:100AFC00D8A0053C015E0650D8A0063C025E063428
:100B0C000E10010B0D26D8B00C2AD8B4082AD8A484
:100B1C0097EF05F008320C320D32032AD8B4AAEF45
:100B2C0005F00AAE089E0850026E0C50016E0D5076
:100B3C00006EB2EF05F0010EACDEB2EF05F0020E66
:100B4C001EEC00F0B2EF05F0040E12EC00F0B2EF68
:0A0B5C0005F0080E25EC00F0120071
:100B660001019C51390806E3300E9C5D03E3010E3A
:080B7600006E01D0006A1200BC
:100B7E000A6A0350D8A40A800750D8A40A820A50E1
:100B8E00D8B422EF06F0030AD8B4DBEF05F00AB0B2
:100B9E00D6EF05F006AE20EF06F01EEF06F002AE21
:100BAE001EEF06F020EF06F00250800B0A6E029E3A
:100BBE000650800B069E0A18D8B4ECEF05F00A50CA
:100BCE00D8B41EEF06F020EF06F00750035CD8B441
:100BDE00F6EF05F0D8A012EF06F018EF06F006506B
:100BEE00025CD8B400EF06F0D8A012EF06F018EFB2
:100BFE0006F00550015CD8B40AEF06F0D8A012EF4B
:100C0E0006F018EF06F00450005CD8B422EF06F0A0
:100C1E00D8B018EF06F00A52D8B420EF06F01EEF47
:100C2E0006F00A52D8B41EEF06F020EF06F0D88078
:0E0C3E001200D8901200D880D8841200120044
:100C4C000B6A0C6A0A6A086A0350D8B4AEEF06F055
:100C5C00028E9E0E035E03BE39EF06F0D8B439EF58
:100C6C0006F09EEF06F0036C080E035CD8A06BEF49
:100C7C0006F0036E083600C008F001C000F002C098
:100C8C0001F0026A080E035CD8A06BEF06F0036E4D
:100C9C00083600C008F001C000F0016A080E035CC1
:100CAC00D8A06BEF06F0036E083600C008F0006A9F
:100CBC00080E035CD8A06BEF06F0036E0836086ACA
:100CCC000350D8A4D89077EF06F00350D8B477EF40
:100CDC0006F0D8900232013200320832032E6FEF48
:100CEC0006F00BBC08A088EF06F0D8A088EF06F041
:100CFC00082AD8B4002AD8B4012AD8B4022A02BED1
:100D0C00B2EF06F00AAEAEEF06F0021E011E001E98
:100D1C00081E082AD8B4002AD8B4012AD8B4022A4A
:100D2C00AEEF06F0026A016A006A086AAEEF06F0DE
:100D3C000B800BAEB7EF06F0026A0AAEB7EF06F007
:100D4C00026E016E006E086E0A360232B7EF06F0C4
:100D5C00000E0C6AB8EF06F0010E0C6E83DDB8EFD6
:100D6C0006F0FF0E0250036E0150026E0050016E31
:060D7C000850006E120099
:100D8200F250026EF29E0500FF6A0150FE6E0050A4
:080D9200FD6E02BEF28E12009C
:100D9A00800E01019C19006E800E000A005CD8B01A
:100DAA006DD19C510008016E01C09CF1800E0118A2
:100DBA00006E800E6E0A005CD8A0C0D0640E046E6D
:100DCA009CC100F039EC01F0120E0024056E000EF1
:100DDA0000BEFF0E066E000E062205C000F006C019
:100DEA0001F0000E06BEFF0E026E036E0036009082
:100DFA0001360236033600360090013602360336D3
:100E0A004F0E0024F66E480E0120F76E000E0220E7
:100E1A00F86E0900F5CF9DF10900F5CF9EF10900A2
:100E2A00F5CF9FF10900F5CFA0F1640E046E9CC1C5
:100E3A0000F039EC01F008C000F00A0E046E39EC3B
:100E4A0001F0090E0024056E000E00BEFF0E066EAC
:100E5A00000E062205C000F006C001F0000E06BE14
:100E6A00FF0E026E036E003600900136023603361C
:100E7A00003600900136023603364F0E0024F66E15
:100E8A00480E0120F76E000E0220F86E0900F5CF19
:100E9A0000F00900F5CF01F00900F5CF02F00900D2
:100EAA00F5CF03F09DC104F09EC105F09FC106F085
:100EBA00A0C107F088EC01F000C09DF101C09EF1CD
:100ECA0002C09FF103C0A0F10A0E046E9CC100F09B
:100EDA0039EC01F008C000F000C001F0000E00BEBD
:100EEA00FF0E026E036E046E01360190023603365F
:100EFA000436013601900236033604364F0E0124B9
:100F0A00F66E480E0220F76E000E0320F86E0900F6
:100F1A00F5CF00F00900F5CF01F00900F5CF02F096
:100F2A000900F5CF03F09DC104F09EC105F09FC1F1
:100F3A0006F0A0C107F088EC01F007D2800E0A0A79
:100F4A00006E800E9C19005C71E20A0E046E9CC150
:100F5A0000F039EC01F0090E0024056E000E00BE07
:100F6A00FF0E066E000E062205C000F006C001F054
:100F7A00000E06BEFF0E026E036E003600900136AA
:100F8A0002360336003600900136023603364F0E1B
:100F9A000024F66E480E0120F76E000E0220F86E4D
:100FAA000900F5CF9DF10900F5CF9EF10900F5CFB3
:100FBA009FF10900F5CFA0F10A0E046E9CC100F062
:100FCA0039EC01F008C000F000C001F0000E00BECC
:100FDA00FF0E026E036E046E01360190023603366E
:100FEA000436013601900236033604364F0E0124C8
:100FFA00F66E480E0220F76E000E0320F86E090006
:10100A00F5CF00F00900F5CF01F00900F5CF02F0A5
:10101A000900F5CF03F09DC104F09EC105F09FC100
:10102A0006F0A0C107F088EC01F08FD19CC100F056
:10103A00000E9CBFFF0E016E026E036E003600901A
:10104A000136023603360036009001360236033680
:10105A004F0E0024F66E480E0120F76E000E022095
:10106A00F86E0900F5CF00F00900F5CF01F009008C
:10107A00F5CF02F00900F5CF03F067D1800E9C1975
:10108A00006E800E6E0A005CD8A0C0D0640E046E9A
:10109A009CC100F039EC01F0120E0024056E000E1E
:1010AA0000BEFF0E066E000E062205C000F006C046
:1010BA0001F0000E06BEFF0E026E036E00360090AF
:1010CA000136023603360036009001360236033600
:1010DA00830E0024F66E480E0120F76E000E0220E1
:1010EA00F86E0900F5CF9DF10900F5CF9EF10900D0
:1010FA00F5CF9FF10900F5CFA0F1640E046E9CC1F3
:10110A0000F039EC01F008C000F00A0E046E39EC68
:10111A0001F0090E0024056E000E00BEFF0E066ED9
:10112A00000E062205C000F006C001F0000E06BE41
:10113A00FF0E026E036E0036009001360236033649
:10114A0000360090013602360336830E0024F66E0E
:10115A00480E0120F76E000E0220F86E0900F5CF46
:10116A0000F00900F5CF01F00900F5CF02F00900FF
:10117A00F5CF03F09DC104F09EC105F09FC106F0B2
:10118A00A0C107F088EC01F000C09DF101C09EF1FA
:10119A0002C09FF103C0A0F10A0E046E9CC100F0C8
:1011AA0039EC01F008C000F000C001F0000E00BEEA
:1011BA00FF0E026E036E046E01360190023603368C
:1011CA00043601360190023603360436830E0124B2
:1011DA00F66E480E0220F76E000E0320F86E090024
:1011EA00F5CF00F00900F5CF01F00900F5CF02F0C4
:1011FA000900F5CF03F09DC104F09EC105F09FC11F
:10120A0006F0A0C107F088EC01F09FD0800E0A0A10
:10121A00006E800E9C19005C71E20A0E046E9CC17D
:10122A0000F039EC01F0090E0024056E000E00BE34
:10123A00FF0E066E000E062205C000F006C001F081
:10124A00000E06BEFF0E026E036E003600900136D7
:10125A000236033600360090013602360336830E14
:10126A000024F66E480E0120F76E000E0220F86E7A
:10127A000900F5CF9DF10900F5CF9EF10900F5CFE0
:10128A009FF10900F5CFA0F10A0E046E9CC100F08F
:10129A0039EC01F008C000F000C001F0000E00BEF9
:1012AA00FF0E026E036E046E01360190023603369B
:1012BA00043601360190023603360436830E0124C1
:1012CA00F66E480E0220F76E000E0320F86E090033
:1012DA00F5CF00F00900F5CF01F00900F5CF02F0D3
:1012EA000900F5CF03F09DC104F09EC105F09FC12E
:1012FA0006F0A0C107F088EC01F027D09CC100F0ED
:10130A00000E9CBFFF0E016E026E036E0036009047
:10131A0001360236033600360090013602360336AD
:10132A00830E0024F66E480E0120F76E000E02208E
:10133A00F86E0900F5CF00F00900F5CF01F00900B9
:0C134A00F5CF02F00900F5CF03F012000F
:1013560001019CBF02D08A9E01D08A8E9CBD02D01C
:101366008A9C01D08A8C9CBB02D08A9A01D08A8A38
:101376009CB902D08A9801D08A8810B102D08A849A
:1013860001D08A948A867FEC04F08A969CB702D0B4
:101396008A9E01D08A8E9CB502D08A9C01D08A8C06
:1013A6009CB302D08A9A01D08A8A9CB102D08A98CC
:1013B60001D08A8810B102D08A8401D08A948A86A4
:1013C6007FEC04F08A9610A103D084EC04F002D0DE
:0613D6008DEC04F0120092
:1013DC0003500718D8A402EF0AF002500618D8A43C
:1013EC0002EF0AF001500518D8A402EF0AF00050E1
:0E13FC000418D8B4D8841200D894120012003D
:08140A00067E27EC02F012003F
:101412006E0E01019C5DD8A0CAD0640E046E9CC100
:1014220000F018EC02F0120E0024056E066A000E9F
:10143200062205C000F006C001F0000E06BEFF0E37
:10144200026E036E00360090013602360336003615
:1014520000900136023603364F0E0024F66E480E17
:101462000120F76E000E0220F86E0900F5CF00F0A1
:101472000900F5CF01F00900F5CF02F00900F5CF20
:1014820003F0000E046E000E056E000E066E7E0E58
:10149200076E88EC01F000C09DF101C09EF102C010
:1014A2009FF103C0A0F1640E046E9CC100F018EC21
:1014B20002F008C000F00A0E046E18EC02F0090EE9
:1014C2000024056E066A000E062205C000F006C062
:1014D20001F0000E06BEFF0E026E036E0036009093
:1014E20001360236033600360090013602360336E4
:1014F2004F0E0024F66E480E0120F76E000E0220F9
:10150200F86E0900F5CF00F00900F5CF01F00900EF
:10151200F5CF02F00900F5CF03F09DC104F09EC1A2
:1015220005F09FC106F0A0C107F088EC01F000C0F1
:101532009DF101C09EF102C09FF103C0A0F10A0E0D
:10154200046E9CC100F018EC02F008C000F000C06C
:1015520001F0000E026E036E046E01360190023637
:1015620003360436013601900236033604364F0E36
:101572000124F66E480E0220F76E000E0320F86E6C
:101582000900F5CF00F00900F5CF01F00900F5CF11
:1015920002F00900F5CF03F09DC104F09EC105F0F1
:1015A2009FC106F0A0C107F088EC01F0B1D09C51B8
:1015B2000A08D8B07ED00A0E046E9CC100F018EC66
:1015C20002F0090E0024056E066A000E062205C00E
:1015D20000F006C001F0000E06BEFF0E026E036EA2
:1015E200003600900136023603360036009001368E
:1015F200023603364F0E0024F66E480E0120F76EB7
:10160200000E0220F86E0900F5CF00F00900F5CFB8
:1016120001F00900F5CF02F00900F5CF03F0000E4A
:10162200046E000E056E000E066E7E0E076E88ECCE
:1016320001F000C09DF101C09EF102C09FF103C004
:10164200A0F10A0E046E9CC100F018EC02F008C072
:1016520000F000C001F0000E026E036E046E01364F
:101662000190023603360436013601900236033603
:1016720004364F0E0124F66E480E0220F76E000E5D
:101682000320F86E0900F5CF00F00900F5CF01F054
:101692000900F5CF02F00900F5CF03F09DC104F077
:1016A2009EC105F09FC106F0A0C107F088EC01F0D1
:1016B2002FD09CC100F0000E016E026E036E003648
:1016C20000900136023603360036009001360236AB
:1016D20003364F0E0024F66E480E0120F76E000E00
:1016E2000220F86E0900F5CF00F00900F5CF01F0F5
:1016F2000900F5CF02F00900F5CF03F0000E046EE9
:10170200000E056E000E066E7E0E076E88EC01F06E
:021712001200C3
:101714000B6A0A6A096A086A0E6A033408360450B6
:10172400085E0550D8A0053C095E0650D8A0063CCA
:101734000A5E0750D8A0073C0B5EE86AD8A0010EE9
:101744000E5E0336070E0C6E0334083609360A366D
:101754000B360E36045003A012D0085E0550D8A0F4
:10176400053C095E0650D8A0063C0A5E0750D8A086
:10177400073C0B5EE86AD8A0010E0E5E11D0082665
:101784000550D8B0053C09260650D8B0063C0A26B8
:101794000750D8B0073C0B26E86AD8B0010E0E26D5
:1017A40003360C2ED1D70234083609360A360B36E6
:1017B4000E36045003A012D0085E0550D8A0053C94
:1017C400095E0650D8A0063C0A5E0750D8A0073C24
:1017D4000B5EE86AD8A0010E0E5E11D008260550F3
:1017E400D8B0053C09260650D8B0063C0A26075056
:1017F400D8B0073C0B26E86AD8B0010E0E26023694
:10180400070E0C6E0234083609360A360B360E36CD
:10181400045002A012D0085E0550D8A0053C095E11
:101824000650D8A0063C0A5E0750D8A0073C0B5EC1
:10183400E86AD8A0010E0E5E11D008260550D8B073
:10184400053C09260650D8B0063C0A260750D8B0F5
:10185400073C0B26E86AD8B0010E0E2602360C2E81
:10186400D1D70134083609360A360B360E36045001
:1018740002A012D0085E0550D8A0053C095E0650AF
:10188400D8A0063C0A5E0750D8A0073C0B5EE86A65
:10189400D8A0010E0E5E11D008260550D8B0053C24
:1018A40009260650D8B0063C0A260750D8B0073C93
:1018B4000B26E86AD8B0010E0E260136070E0C6E10
:1018C4000134083609360A360B360E36045001A0A8
:1018D40012D0085E0550D8A0053C095E0650D8A079
:1018E400063C0A5E0750D8A0073C0B5EE86AD8A005
:1018F400010E0E5E11D008260550D8B0053C09260D
:101904000650D8B0063C0A260750D8B0073C0B2630
:10191400E86AD8B0010E0E2601360C2ED1D7003459
:10192400083609360A360B360E36045001A012D09A
:10193400085E0550D8A0053C095E0650D8A0063CB8
:101944000A5E0750D8A0073C0B5EE86AD8A0010ED7
:101954000E5E11D008260550D8B0053C0926065065
:10196400D8B0063C0A260750D8B0073C0B26E86AD4
:10197400D8B0010E0E260036070E0C6E0034083661
:1019840009360A360B360E36045000A012D0085E13
:101994000550D8A0053C095E0650D8A0063C0A5E56
:1019A4000750D8A0073C0B5EE86AD8A0010E0E5E73
:1019B40011D008260550D8B0053C09260650D8B0E9
:1019C400063C0A260750D8B0073C0B26E86AD8B074
:1019D400010E0E2600360C2ED1D700B00ED00450C6
:1019E40008260550D8B0053C09260650D8B0063C58
:0C19F4000A260750D8B0073C0B26120052
:101A00000B6A0A6A096A00500402F4CF09F0F3CFA6
:101A100008F001500502F4CF0BF0F3CF0AF00050AC
:101A20000502F3500926F4500A22E86A0B220150FD
:101A30000402F3500926F4500A22E86A0B2208C077
:101A400000F009C001F00AC002F00BC003F0120060
:101A50000B6A0C6A086A0350D8B4ACEF0DF002C0F0
:101A60000AF0028E9E0E035E03AE9CEF0DF0036C37
:101A7000080E035CD8A069EF0DF0036E083600C0B5
:101A800008F001C000F002C001F0026A080E035C19
:101A9000D8A069EF0DF0036E083600C008F001C051
:101AA00000F0016A080E035CD8A069EF0DF0036E28
:101AB000083600C008F0006A080E035CD8A069EF81
:101AC0000DF0036E0836086A0350D8A4D89075EF5D
:101AD0000DF00350D8B475EF0DF0D89002320132FA
:101AE00000320832032E6DEF0DF00BBC08A086EF1C
:101AF0000DF0D8A086EF0DF0082AD8B4002AD8B48B
:101B0000012AD8B4022A02BEB0EF0DF00AAEACEF43
:101B10000DF0021E011E001E081E082AD8B4002A5D
:101B2000D8B4012AD8B4022AACEF0DF0026A016AD7
:101B3000006A086AACEF0DF00B800BAEB7EF0DF04A
:101B4000026A0AAEB7EF0DF0026E016E006E086E0B
:101B50000A360232B7EF0DF00C6A000EB8EF0DF046
:101B6000010E0C6E000E38EC04F0B8EF0DF0FF0E15
:101B70000250036E0150026E0050016E0850006E5C
:021B8000120051
:101B82000050086E0150006E0250016E0350026E4A
:101B9200036A0B6A0C6A9E0E036E0A6A020E0C6ED0
:061BA20032EC00F012001D
:101BA8000C6A0E6A0250D8A4EDEF0DF001C002F0E5
:101BB80000C001F0006A0E860250D8A4EDEF0DF0C7
:101BC80001C002F0016A0E960E880250D8B4FFEFE9
:101BD8000DF00E50035ED8A4D8A005EF0EF0D890F3
:101BE80002BE0BEF0EF0003601360236032EF4EF7C
:101BF8000DF005EF0EF0010E0C6E1EEC00F00FEF6D
:101C08000EF0020E0C6E25EC00F00FEF0EF0040E35
:081C18000C6E0EEC00F012004E
:101C20000101946B956B886B896B76C100F077C16D
:101C300001F078C102F0010E7627000E7723782399
:101C400000C0F6FF01C0F7FF02C0F8FF0900F5CFA2
:101C500000F000C085F10052D8B41CEF1EF0855191
:101C6000250A0BE074C1E1FF75C1E2FF85C1E6FF03
:101C7000744B752B944B952BD8D7866B876B886BE1
:101C8000896B23D08887010E7627000E772378236F
:101C900059D08881010E7627000E7723782352D001
:101CA0008883010E7627000E772378234BD089870F
:101CB000010E7627000E7723782344D08885010E05
:101CC0007627000E772378233DD076C1F6FF77C1C3
:101CD000F7FF78C1F8FF0900F5CF01F001502D0A98
:101CE000D1E076C1F6FF77C1F7FF78C1F8FF0900B0
:101CF000F5CF01F00150200ACCE076C1F6FF77C1A4
:101D0000F7FF78C1F8FF0900F5CF01F001502B0A69
:101D1000C7E076C1F6FF77C1F7FF78C1F8FF090089
:101D2000F5CF01F00150230AC2E076C1F6FF77C17A
:101D3000F7FF78C1F8FF0900F5CF01F00150300A34
:101D4000BDE001D09ED788A301D0889188A701D09B
:101D5000889576C1F6FF77C1F7FF78C1F8FF0900D3
:101D6000F5CF00F0000E016E00C09CF1B3EC05F061
:101D7000005235E0866B876B86C100F087C101F0A9
:101D80000A0E046E000E056E3BDE76C1F6FF77C1CB
:101D9000F7FF78C1F8FF0900F5CF02F002500024E8
:101DA000866F000E0120876F300E865F000E875B06
:101DB000010E7627000E7723782376C1F6FF77C1D0
:101DC000F7FF78C1F8FF0900F5CF00F0000E016EB3
:101DD00000C09CF1B3EC05F00052CEE133D076C1E7
:101DE000F6FF77C1F7FF78C1F8FF0900F5CF01F0E2
:101DF00001502A0A27E179C1E9FF7AC1EAFFEECF53
:101E000000F0EECF01F000C0E9FF01C0EAFFEECF25
:101E100086F1EECF87F179C1E9FF7AC1EAFF020EC0
:101E2000EE24006E000EEE20016E79C1E1FF7AC152
:101E3000E2FF00C0E6FF01C0E6FF010E7627000EBC
:101E40007723782376C1F6FF77C1F7FF78C1F8FFD3
:101E50000900F5CF01F001502E0A6FE1010E76273F
:101E6000000E7723782376C1F6FF77C1F7FF78C19C
:101E7000F8FF0900F5CF01F001502A0A28E179C1E5
:101E8000E9FF7AC1EAFFEECF00F0EECF01F000C02B
:101E9000E9FF01C0EAFFEECF83F1EECF84F179C113
:101EA000E9FF7AC1EAFF020EEE24006E000EEE207A
:101EB000016E79C1E1FF7AC1E2FF00C0E6FF01C017
:101EC000E6FF010E7627000E7723782335D0836B4B
:101ED000846B76C1F6FF77C1F7FF78C1F8FF090080
:101EE000F5CF00F0000E016E00C09CF1B3EC05F0E0
:101EF000005222E083C100F084C101F00A0E046E9A
:101F0000000E056E7DDD76C1F6FF77C1F7FF78C163
:101F1000F8FF0900F5CF02F002500024836F000E95
:101F20000120846F300E835F000E845B010E7627E4
:101F3000000E77237823CDD703D0836B846B8989F8
:101F400076C100F077C101F078C102F0010E76276A
:101F5000000E7723782300C0F6FF01C0F7FF02C010
:101F6000F8FF0900F5CF85F1F9D094C100F095C1D3
:101F700001F020EF1EF08889E3D789852ED1888B68
:101F800089812BD1898329D1888D27D126D1888B2E
:101F9000888F23D179C1E9FF7AC1EAFFEECF00F043
:101FA000EECF01F000C0E9FF01C0EAFFEECF90F1F3
:101FB000EECF91F179C1E9FF7AC1EAFF020EEE247A
:101FC000006E000EEE20016E79C1E1FF7AC1E2FFE2
:101FD00000C0E6FF01C0E6FF000E911902E1000E0D
:101FE000901904E16E0E906F000E916F926B936BDF
:101FF00092519025E96E93519121EA6EEE520BE0D9
:10200000010E9225006E000E9321016E00C092F128
:1020100001C093F1EDD7835184110AE09351845D9F
:1020200002E19251835D04E283C192F184C193F194
:102030008751935D02E18651925D05E29251865F80
:102040009351875B02D0866B876B88B716D086C1A9
:1020500000F087C101F0010E865F000E875B005023
:1020600001100BE074C1E1FF75C1E2FF200EE66EC6
:10207000744B752B944B952BEAD792C102F093C108
:1020800003F0010E925D006E000E9359016E00C0C8
:1020900092F101C093F10250031019E090C1E9FFE1
:1020A00091C1EAFF74C1E1FF75C1E2FFEECFE6FF27
:1020B000744B752B010E9025006E000E9121016E60
:1020C00000C090F101C091F1944B952BD6D788A711
:1020D00016D086C100F087C101F0010E865F000EA8
:1020E000875B005001100BE074C1E1FF75C1E2FF96
:1020F000200EE66E744B752B944B952BEAD795D535
:1021000079C1E9FF7AC1EAFFEECF00F0EECF01F02E
:1021100000C0E9FF01C0EAFFEECF85F179C1E9FF18
:102120007AC1EAFF020EEE24006E000EEE20016E70
:1021300079C1E1FF7AC1E2FF00C0E6FF01C0E6FF1E
:10214000850E906F010E916F010E926F000E936FCE
:1021500062D7C00E8813000E89133FD08551000A44
:10216000D8B403D785516C0AD8B405D785514C0A29
:10217000D8B401D78551660AD8B4FFD68551450A2F
:10218000D8B4FDD68551650AD8B4FAD68551670A08
:10219000D8B4F8D685516F0AD8B4F6D68551640AFA
:1021A000D8B4F4D68551690AD8B4F0D68551700AEE
:1021B000D8B4EDD68551580AD8B4E9D68551780AF5
:1021C000D8B4E6D68551730AD8B4E4D68551630AEB
:1021D00097E08551750ABDE0B3D7000E8815006EF3
:1021E0008951070B016E00500110D8B4C3EF19F0EC
:1021F00089A904D0060E836F000E846F79C1E9FFB0
:102200007AC1EAFFEECF00F0EECF01F000C0E9FFA7
:1022100001C0EAFFEECF8AF1EECF8BF1EECF8CF169
:10222000EECF8DF179C1E9FF7AC1EAFF040EEE2409
:10223000006E000EEE20016E79C1E1FF7AC1E2FF6F
:1022400000C0E6FF01C0E6FF046A056A066A076A85
:102250008AC100F08BC101F08CC102F08DC103F086
:10226000BFEC05F0010ED8B0000E006E005205E084
:102270008C7F030E8813000E89138E6B8F6B8AC1BF
:1022800000F08BC101F08CC102F08DC103F0046A33
:10229000056A066A076AEEEC09F0000ED8A4010E82
:1022A000006E0052D8B48AD08DC100F0016A026A73
:1022B000036AFF0E0016000E01167E0E005E000E71
:1022C000015A00C08EF101C08FF1010E005E000EB8
:1022D000015A00C08EF101C08FF1030E046E000E92
:1022E000056E00EC0DF000C08EF101C08FF10A0EFA
:1022F000046E000E056E93EC04F000C08EF101C078
:102300008FF1800E0118026E800E025C02E1000E59
:10231000005C05E2010E01018E5F000E8F5B010182
:102320008E5100089C6FCDEC06F08AC104F08BC181
:1023300005F08CC106F08DC107F088EC01F000C0FB
:1023400090F101C091F102C092F103C093F1000E2F
:10235000046E000E056E000E066E7F0E076E90C1B5
:1023600000F091C101F092C102F093C103F0BFEC03
:1023700005F0010ED8B0000E006E005205E0010E0F
:102380008E5F000E8F5B1AD0000E046E000E056E7D
:10239000200E066E820E076E90C100F091C101F012
:1023A00092C102F093C103F0BFEC05F0000ED8B06B
:1023B000010E006E005202E08E4B8F2B800E006EDD
:1023C000800E8F19005C02E18E51000803E3010EBC
:1023D000856F02D08EC185F189B118D089A315D03F
:1023E000800E8F19006E7F0E005C02E1FC0E8E5D88
:1023F0000BE3800E8F19006E800E8419005C02E1E1
:1024000083518E5D01E201D001D0EFD3835184115D
:1024100006E089A304D0010E835F000E845B845123
:10242000000802E18351080803E2080E856F02D01C
:1024300083C185F18AC100F08BC101F08CC102F02B
:102440008DC103F0046A056A066A076AEEEC09F0BA
:10245000000ED8A4010E006E0052D8B44BD18EC12C
:102460009CF1CDEC06F000C004F001C005F002C004
:1024700006F003C007F08AC100F08BC101F08CC1E7
:1024800002F08DC103F0F6EC04F000C08AF101C047
:102490008BF102C08CF103C08DF101018551000860
:1024A0009C6FCDEC06F000C004F001C005F002C046
:1024B00006F003C007F08AC100F08BC101F08CC1A7
:1024C00002F08DC103F0F6EC04F000C096F101C0FB
:1024D00097F102C098F103C099F196C18AF197C1B2
:1024E0008BF198C18CF199C18DF196C100F097C123
:1024F00001F098C102F099C103F026EC06F0C1EC9E
:102500000DF000C004F001C005F002C006F003C0E9
:1025100007F096C100F097C101F098C102F099C18F
:1025200003F005EC0AF0000E046E000E056E000EBE
:10253000066E7E0E076EBFEC05F0000ED8B0010EE1
:10254000006E00521AE08AC100F08BC101F08CC10C
:1025500002F08DC103F0000E046E000E056E000E39
:10256000066E7E0E076E27EC02F000C08AF101C0F5
:102570008BF102C08CF103C08DF18AC100F08BC1D8
:1025800001F08CC102F08DC103F026EC06F00101D0
:102590008551010F096E0A6A000E0A2209C004F073
:1025A0000AC005F0000E0ABEFF0E066E076E043666
:1025B000049005360636073604360490053606368E
:1025C00007369B0E0424F66E490E0520F76E000EAA
:1025D0000620F86E0900F5CF05F00900F5CF06F0EA
:1025E0000900F5CF07F00900F5CF08F00850035CAB
:1025F00008E10750025C05E10650015C02E105506C
:10260000005C1EE301018AC100F08BC101F08CC1A6
:1026100002F08DC103F0CD0E046ECC0E056E4C0E93
:10262000066E7B0E076E88EC01F000C08AF101C0D7
:102630008BF102C08CF103C08DF18E4B8F2B5AD0E1
:102640008AC100F08BC101F08CC102F08DC103F092
:1026500026EC06F085C104F0000E056E066E076ECE
:1026600004360490053606360736043604900536DF
:10267000063607369B0E0424F66E490E0520F76ECB
:10268000000E0620F86E0900F5CF05F00900F5CF21
:1026900006F00900F5CF07F00900F5CF08F0085063
:1026A000035C08E10750025C05E10650015C02E1B1
:1026B0000550005C1FE201018AC100F08BC101F0EE
:1026C0008CC102F08DC103F0000E046E000E056E89
:1026D000200E066E820E076E88EC01F000C08AF1B3
:1026E00001C08BF102C08CF103C08DF1010E8E5F31
:1026F000000E8F5B010189A393D089B791D0800E22
:10270000000A006E800E8419005C02E183510A0801
:1027100004E20A0E836F000E846F8AC100F08BC141
:1027200001F08CC102F08DC103F026EC06F000C070
:1027300090F101C091F102C092F103C093F1905168
:1027400091119211931142E00A0E046E000E056E73
:10275000066E076E90C100F091C101F092C102F0C7
:1027600093C103F08AEC0BF008C000F009C001F03F
:102770000AC002F00BC003F0000E046E031808E15B
:102780000450021805E10450011802E10050000A4B
:102790001DE1010E835F000E845B0A0E046E000EC5
:1027A000056E066E076E90C100F091C101F092C1F6
:1027B00002F093C103F08AEC0BF000C090F101C06D
:1027C00091F102C092F103C093F1B9D7800E841940
:1027D000006E800E005C02E18551835D21E2835131
:1027E000855D9C6FCDEC06F000C004F001C005F0E3
:1027F00002C006F003C007F08AC100F08BC101F0EF
:102800008CC102F08DC103F0F6EC04F000C08AF137
:1028100001C08BF102C08CF103C08DF183C185F141
:10282000050E01018325006E000E8421016E00500B
:10283000865F0150875B8351841103E189B701D022
:1028400004D0010E865F000E875B030E8815006EB4
:1028500089C101F0000E01160050011004E0010EC4
:10286000865F000E875B88A539D088A312D088A127
:1028700003D02D0E7B6F02D02B0E7B6F74C1E1FF56
:1028800075C1E2FF7BC1E6FF744B752B944B952B12
:102890000CD088A10AD074C1E1FF75C1E2FF200EFF
:1028A000E66E744B752B944B952B800E006E800E4C
:1028B0008719005C02E1865100080FE274C1E1FF54
:1028C00075C1E2FF300EE66E744B752B944B952B61
:1028D000010E865F000E875BE8D73AD088B718D024
:1028E000800E006E800E8719005C02E186510008A0
:1028F0000FE274C1E1FF75C1E2FF200EE66E744B7A
:10290000752B944B952B010E865F000E875BE8D7E5
:1029100088A312D088A103D02D0E7C6F02D02B0E7D
:102920007C6F74C1E1FF75C1E2FF7CC1E6FF744BAF
:10293000752B944B952B0CD088A10AD074C1E1FF64
:1029400075C1E2FF200EE66E744B752B944B952BF0
:102950008AC100F08BC101F08CC102F08DC103F07F
:1029600026EC06F000C090F101C091F102C092F196
:1029700003C093F185C100F0000E016E026E036E7C
:1029800000360090013602360336003600900136DC
:10299000023603369B0E0024F66E490E0120F76EB8
:1029A000000E0220F86E0900F5CF04F00900F5CF03
:1029B00005F00900F5CF06F00900F5CF07F090C14A
:1029C00000F091C101F092C102F093C103F08AECD2
:1029D0000BF0300E002674C1E1FF75C1E2FF00C0AC
:1029E000E6FF744B752B944B952B8351841103E1B7
:1029F00089B701D06FD074C1E1FF75C1E2FF2E0E1F
:102A0000E66E744B752B944B952B8551835F000EAE
:102A1000845B85534DE0850785C100F0000E016E93
:102A2000026E036E00360090013602360336003621
:102A300000900136023603369B0E0024F66E490ED6
:102A40000120F76E000E0220F86E0900F5CF04F0A9
:102A50000900F5CF05F00900F5CF06F00900F5CF24
:102A600007F090C100F091C101F092C102F093C152
:102A700003F08AEC0BF00A0E046E000E056E066E73
:102A8000076E8AEC0BF008C000F009C001F00AC024
:102A900002F00BC003F0300E002674C1E1FF75C1D7
:102AA000E2FF00C0E6FF744B752B944B952BB1D71A
:102AB000835184110FE074C1E1FF75C1E2FF300E54
:102AC000E66E744B752B944B952B010E835F000EB5
:102AD000845BEED788AB0BD074C1E1FF75C1E2FF18
:102AE000450EE66E744B752B944B952B0AD074C132
:102AF000E1FF75C1E2FF650EE66E744B752B944BDA
:102B0000952B800E8F19006E800E005C02E1000E86
:102B10008E5D11E28E5100088E6F8F51000E8F571F
:102B200074C1E1FF75C1E2FF2D0EE66E744B752B8B
:102B3000944B952B0AD074C1E1FF75C1E2FF2B0EB7
:102B4000E66E744B752B944B952B0A0E046E000E9B
:102B5000056E8EC100F08FC101F093EC04F0300ED1
:102B6000002674C1E1FF75C1E2FF00C0E6FF01016C
:102B7000744B752B944B952B0A0E046E000E056E4C
:102B80008EC100F08FC101F093EC04F008C000F09A
:102B900009C001F0300E002674C1E1FF75C1E2FFEB
:102BA00000C0E6FF0101744B752B944B952B88A751
:102BB0001AD0800E006E800E8719005C02E18651EB
:102BC000000811E274C1E1FF75C1E2FF200EE66E5C
:102BD000744B752B944B952B010E865F000E875B13
:102BE00086518711EFE115EF0EF089A3F3D0800E27
:102BF0008F19006E800E005C02E1000E8E5D0AE20D
:102C0000010E8E5D006E000E8F59016E0050835FC5
:102C10000150845B8AC100F08BC101F08CC102F0CD
:102C20008DC103F026EC06F000C090F101C091F1D7
:102C300002C092F103C093F1010E856F85510A0A1B
:102C400034E085C100F0000E016E026E036E0036A6
:102C50000090013602360336003600900136023607
:102C600003369B0E0024F66E490E0120F76E000E0F
:102C70000220F86E0900F5CF01F00900F5CF02F04F
:102C80000900F5CF03F00900F5CF04F00450935D7F
:102C900008E10350925D05E10250915D02E10150AF
:102CA000905D01E202D0852BC9D78551835D9A6F73
:102CB000000E84599B6F9AC183F19BC184F190C12E
:102CC00000F091C101F092C102F093C103F0C1EC98
:102CD0000DF000C004F001C005F002C006F003C012
:102CE00007F08AC100F08BC101F08CC102F08DC1E8
:102CF00003F005EC0AF000C096F101C097F102C0A4
:102D000098F103C099F19AC19CF1CDEC06F096C1FF
:102D100004F097C105F098C106F099C107F088EC5E
:102D200001F0000E046E000E056E000E066E7E0EA3
:102D3000076E27EC02F026EC06F000C090F101C00F
:102D400091F102C092F103C093F18351841142E0EA
:102D50000A0E046E000E056E066E076E90C100F03E
:102D600091C101F092C102F093C103F08AEC0BF023
:102D700008C000F009C001F00AC002F00BC003F067
:102D8000000E046E031808E10450021805E1045017
:102D9000011802E10050000A1DE10A0E046E000E47
:102DA000056E066E076E90C100F091C101F092C1F0
:102DB00002F093C103F08AEC0BF000C090F101C067
:102DC00091F102C092F103C093F1010E835F000EF6
:102DD000845BBBD7800E006E800E8419005C02E11C
:102DE00083510C0816E383C19CF109EC0AF08AC1F7
:102DF00004F08BC105F08CC106F08DC107F027EC03
:102E000002F000C08AF101C08BF102C08CF103C056
:102E10008DF18AC100F08BC101F08CC102F08DC12F
:102E200003F0046A056A066A076AEEEC09F0000E10
:102E3000D8A4010E006E0052D8B477D08AC100F039
:102E40008BC101F08CC102F08DC103F026EC06F0BD
:102E5000000E046E031808E10450021805E1045046
:102E6000011802E10050000A60E1800E006E800E41
:102E70008F19005C02E18E51010857E28EC19CF16E
:102E8000CDEC06F000C004F001C005F002C006F071
:102E900003C007F08AC100F08BC101F08CC102F0C1
:102EA0008DC103F0F6EC04F05F0E046E700E056E3B
:102EB000090E066E810E076EBFEC05F0010ED8B04C
:102EC000000E006E005206E0090E01018E5F000E3A
:102ED0008F5B05D00101080E8E5F000E8F5B8EC1E7
:102EE0009CF1CDEC06F000C004F001C005F002C07A
:102EF00006F003C007F08AC100F08BC101F08CC15D
:102F000002F08DC103F0F6EC04F026EC06F000C0F0
:102F100090F101C091F102C092F103C093F101015F
:102F20008A6B8B6B8C6B8D6B38D08AC100F08BC138
:102F300001F08CC102F08DC103F026EC06F000C058
:102F400090F101C091F102C092F103C093F190C1E0
:102F500000F091C101F092C102F093C103F0C1EC05
:102F60000DF000C004F001C005F002C006F003C07F
:102F700007F08AC100F08BC101F08CC102F08DC155
:102F800003F005EC0AF000C08AF101C08BF102C029
:102F90008CF103C08DF18E6B8F6B010E856F8551A7
:102FA0000A0A34E085C100F0000E016E026E036E65
:102FB00000360090013602360336003600900136A6
:102FC000023603369B0E0024F66E490E0120F76E82
:102FD000000E0220F86E0900F5CF01F00900F5CFD0
:102FE00002F00900F5CF03F00900F5CF04F004501A
:102FF000935D08E10350925D05E10250915D02E1AD
:103000000150905D01E202D0852BC9D785518325FF
:10301000006E000E8421016E8E5100268F51012218
:103020000050865F0150875B89B704D083518411BB
:1030300001E104D0010E865F000E875B030E881548
:10304000006E89C101F0000E01160050011004E06D
:10305000010E865F000E875B88A539D088A312D049
:1030600088A103D02D0E7D6F02D02B0E7D6F74C111
:10307000E1FF75C1E2FF7DC1E6FF744B752B944BF8
:10308000952B0CD088A10AD074C1E1FF75C1E2FF75
:10309000200EE66E744B752B944B952B800E006EB4
:1030A000800E8719005C02E1865100080FE274C1AE
:1030B000E1FF75C1E2FF300EE66E744B752B944B49
:1030C000952B010E865F000E875BE8D73AD088B754
:1030D00018D0800E006E800E8719005C02E18651C8
:1030E00000080FE274C1E1FF75C1E2FF200EE66E39
:1030F000744B752B944B952B010E865F000E875BEE
:10310000E8D788A312D088A103D02D0E7E6F02D0FD
:103110002B0E7E6F74C1E1FF75C1E2FF7EC1E6FF39
:10312000744B752B944B952B0CD088A10AD074C18D
:10313000E1FF75C1E2FF200EE66E744B752B944BD8
:10314000952B85C100F0850700524CE085C100F049
:10315000000E016E026E036E0036009001360236DC
:103160000336003600900136023603369B0E0024EB
:10317000F66E490E0120F76E000E0220F86E09006F
:10318000F5CF04F00900F5CF05F00900F5CF06F002
:103190000900F5CF07F090C100F091C101F092C194
:1031A00002F093C103F08AEC0BF00A0E046E000EDD
:1031B000056E066E076E8AEC0BF008C000F009C0C1
:1031C00001F00AC002F00BC003F0300E002674C1FB
:1031D000E1FF75C1E2FF00C0E6FF744B752B944B15
:1031E000952BAFD7800E006E800E8F19005C02E128
:1031F0008E5100080FE274C1E1FF75C1E2FF300E8D
:10320000E66E744B752B944B952B010E8E5F000E62
:103210008F5BE8D7800E000A006E800E8419005C78
:1032200002E18351080803E2080E856F02D083C1D2
:1032300085F18551835F000E845B855303E189B777
:1032400001D00AD074C1E1FF75C1E2FF2E0EE66E17
:10325000744B752B944B952B85C19CF1CDEC06F0EE
:103260008AC104F08BC105F08CC106F08DC107F056
:1032700088EC01F028EC0DF000C090F101C091F154
:1032800002C092F103C093F185534DE0850785C1DB
:1032900000F0000E016E026E036E003600900136E3
:1032A00002360336003600900136023603369B0E96
:1032B0000024F66E490E0120F76E000E0220F86E13
:1032C0000900F5CF04F00900F5CF05F00900F5CFAE
:1032D00006F00900F5CF07F090C100F091C101F0B0
:1032E00092C102F093C103F08AEC0BF00A0E046E57
:1032F000000E056E066E076E8AEC0BF008C000F03B
:1033000009C001F00AC002F00BC003F0300E002625
:1033100074C1E1FF75C1E2FF00C0E6FF744B752B7D
:10332000944B952BB1D7835184110FE074C1E1FF09
:1033300075C1E2FF300EE66E744B752B944B952BE6
:10334000010E835F000E845BEED788A71AD0800E33
:10335000006E800E8719005C02E18651000811E2C0
:1033600074C1E1FF75C1E2FF200EE66E744B752B50
:10337000944B952B010E865F000E875B865187115B
:10338000EFE115EF0EF0C00E8815016E89C102F055
:10339000000E0216000E021802E1000E0118D8A459
:1033A00080D088A927D079C1E9FF7AC1EAFFEECFA2
:1033B00000F0EECF01F000C0E9FF01C0EAFFEECF60
:1033C00090F1EECF91F1EECF92F1EECF93F179C182
:1033D000E9FF7AC1EAFF040EEE24006E000EEE2033
:1033E000016E79C1E1FF7AC1E2FF00C0E6FF01C0D2
:1033F000E6FF2FD079C1E9FF7AC1EAFFEECF00F0F6
:10340000EECF01F000C0E9FF01C0EAFFEECF00F00F
:10341000EECF01F0000E01BEFF0E026E036E00C083
:1034200090F101C091F102C092F103C093F179C112
:10343000E9FF7AC1EAFF020EEE24006E000EEE20D4
:10344000016E79C1E1FF7AC1E2FF00C0E6FF01C071
:10345000E6FF800E9319006E800E005C08E1000EFE
:10346000925D05E1000E915D02E1000E905D18E2B3
:10347000030E8813000E8913006A016A026A036A48
:103480009051005E9151015A9251025A9351035A40
:1034900000C090F101C091F102C092F103C093F11C
:1034A0004ED088A927D079C1E9FF7AC1EAFFEECFD3
:1034B00000F0EECF01F000C0E9FF01C0EAFFEECF5F
:1034C00090F1EECF91F1EECF92F1EECF93F179C181
:1034D000E9FF7AC1EAFF040EEE24006E000EEE2032
:1034E000016E79C1E1FF7AC1E2FF00C0E6FF01C0D1
:1034F000E6FF25D079C1E9FF7AC1EAFFEECF00F0FF
:10350000EECF01F000C0E9FF01C0EAFFEECF90F17D
:10351000EECF91F1000E926F936F79C1E9FF7AC1FE
:10352000EAFF020EEE24006E000EEE20016E79C15D
:10353000E1FF7AC1E2FF00C0E6FF01C0E6FF000E36
:10354000841902E1000E83190FE1000E006E931939
:1035500008E10050921905E10050911902E19051E3
:10356000000A02E1834B842BC00E8815006E00C058
:1035700005F0AED0010E856F85510A0A34E085C191
:1035800000F0000E016E026E036E003600900136F0
:1035900002360336003600900136023603369B0EA3
:1035A0000024F66E490E0120F76E000E0220F86E20
:1035B0000900F5CF01F00900F5CF02F00900F5CFC1
:1035C00003F00900F5CF04F00450935D08E10350C7
:1035D000925D05E10250915D02E10150905D01E2D2
:1035E00002D0852BC9D782D0010E856F8551080A7C
:1035F00034E085C100F0000E016E026E036E0036ED
:10360000009001360236033600360090013602364D
:103610000336320E0024F66E4A0E0120F76E000EBD
:103620000220F86E0900F5CF01F00900F5CF02F095
:103630000900F5CF03F00900F5CF04F00450935DC5
:1036400008E10350925D05E10250915D02E10150F5
:10365000905D01E202D0852BC9D748D0010E856F5D
:1036600085510C0A34E085C100F0000E016E026E37
:10367000036E0036009001360236033600360090A5
:10368000013602360336E90E0024F66E480E01209C
:10369000F76E000E0220F86E0900F5CF01F0090068
:1036A000F5CF02F00900F5CF03F00900F5CF04F0E3
:1036B0000450935D08E10350925D05E10250915D75
:1036C00002E10150905D01E202D0852BC9D70ED0F6
:1036D0000550000AD8B44ED70550C00AD8B44AD70E
:1036E0000550800A81E00550400AB8E0800E006E67
:1036F000800E8419005C02E18351855D03E283C181
:1037000085F10DD0800E8419006E800E005C02E100
:103710008551835D04E285C183F1000E846F86517B
:1037200087110EE0030E8815006E89C101F0000EAE
:1037300001160050011004E0010E865F000E875B49
:10374000800E8419006E800E8719005C02E186519C
:10375000835D05E28351865F8451875B02D0866B6F
:10376000876BC40E8815016E8951080B026E0250DA
:10377000080A02E1400E011808E18651871104E0B1
:10378000010E865F000E875B1CD0C00E8815016E8F
:103790008951080B026E0250080A02E1800E0118DE
:1037A00010E1800E006E800E8719005C02E18651E8
:1037B000020805E2020E865F000E875B02D0866B70
:1037C000876B88A55DD088A312D088A103D02D0E69
:1037D0007F6F02D02B0E7F6F74C1E1FF75C1E2FFD6
:1037E0007FC1E6FF744B752B944B952B34D088A189
:1037F0000BD074C1E1FF75C1E2FF200EE66E744B81
:10380000752B944B952B27D0C00E8815016E8951CE
:10381000080B026E0250080A02E1800E01181BE13B
:1038200074C1E1FF75C1E2FF300EE66E744B752B7B
:10383000944B952B88AB03D0580E806F02D0780E36
:10384000806F74C1E1FF75C1E2FF80C1E6FF744B78
:10385000752B944B952B8651871111E074C1E1FFB4
:1038600075C1E2FF300EE66E744B752B944B952BB1
:10387000010E865F000E875B86518711EFE174D0E1
:103880008651871113E088B711D074C1E1FF75C16B
:10389000E2FF200EE66E744B752B944B952B010EB8
:1038A000865F000E875B86518711EFE188A312D0F7
:1038B00088A103D02D0E816F02D02B0E816F74C1B1
:1038C000E1FF75C1E2FF81C1E6FF744B752B944B9C
:1038D000952B0CD088A10AD074C1E1FF75C1E2FF1D
:1038E000200EE66E744B752B944B952BC00E8815ED
:1038F000016E8951080B026E0250080A02E1400E67
:1039000001180BE174C1E1FF75C1E2FF300EE66EF4
:10391000744B752B944B952B27D0C00E8815016ED8
:103920008951080B026E0250080A02E1800E01184C
:103930001BE174C1E1FF75C1E2FF300EE66E744B0E
:10394000752B944B952B88AB03D0580E826F02D009
:10395000780E826F74C1E1FF75C1E2FF82C1E6FF9C
:10396000744B752B944B952B800E006E800E841932
:10397000005C02E18351855D0BE274C1E1FF75C11A
:10398000E2FF300EE66E744B752B944B952BECD703
:1039900083C100F084C101F0010E835F000E845BDF
:1039A00000500110D8B42AD1C00E8815006E00C096
:1039B00096F10AD183C100F084C101F0000E84BFEA
:1039C000FF0E026E036E003600900136023603369B
:1039D000003600900136023603369B0E0024F66E48
:1039E000490E0120F76E000E0220F86E0900F5CF97
:1039F00004F00900F5CF05F00900F5CF06F0090045
:103A0000F5CF07F090C100F091C101F092C102F032
:103A100093C103F08AEC0BF00A0E046E000E056EE3
:103A2000066E076E8AEC0BF008C000F009C001F0CA
:103A30000AC002F00BC003F0300E0024856FD3D013
:103A400088AB45D083C100F084C101F0000E84BF73
:103A5000FF0E026E036E003600900136023603360A
:103A600000360090013602360336320E0024F66E20
:103A70004A0E0120F76E000E0220F86E0900F5CF05
:103A800004F00900F5CF05F00900F5CF06F00900B4
:103A9000F5CF07F090C100F091C101F092C102F0A2
:103AA00093C103F08AEC0BF00F0E0016000E011606
:103AB00002160316DE0E0024F66E4A0E0120F76E83
:103AC000000E0220F86E0900F5CF85F144D083C1C5
:103AD00000F084C101F0000E84BFFF0E026E036E81
:103AE000003600900136023603360036009001366B
:103AF00002360336320E0024F66E4A0E0120F76EAF
:103B0000000E0220F86E0900F5CF04F00900F5CF91
:103B100005F00900F5CF06F00900F5CF07F090C1D8
:103B200000F091C101F092C102F093C103F08AEC60
:103B30000BF00F0E0016000E011602160316CD0E26
:103B40000024F66E4A0E0120F76E000E0220F86E79
:103B50000900F5CF85F147D083C100F084C101F0A1
:103B6000000E84BFFF0E026E036E00360090013619
:103B70000236033600360090013602360336E90E6F
:103B80000024F66E480E0120F76E000E0220F86E3B
:103B90000900F5CF04F00900F5CF05F00900F5CFD5
:103BA00006F00900F5CF07F090C100F091C101F0D7
:103BB00092C102F093C103F08AEC0BF0070E0014DF
:103BC000856F300E85270FD09651000AD8B4F2D6F3
:103BD0009651C00AD8B4EED69651800AD8B430D7E0
:103BE0009651400AB9E074C1E1FF75C1E2FF85C199
:103BF000E6FF744B752B944B952BCAD688A71AD029
:103C0000800E006E800E8719005C02E1865100086C
:103C100011E274C1E1FF75C1E2FF200EE66E744B44
:103C2000752B944B952B010E865F000E875B86519A
:103C30008711EFE115EF0EF094C100F095C101F08E
:023C4000120070
:103C42000EC1E1FF0FC1E2FF74C1E6FF0CC100F03B
:0A3C52000DC101F0C1EC06F01200F4
:103C5C000101109174C19CF1ABEC09F010811200C0
:103C6C00086A096A100E0C6E0134083609360450C5
:103C7C00085E0550D8A0053C095ED8B007D00450AA
:103C8C0008260550D8B0053C0926D89000360136D8
:063C9C000C2EEAD7120015
:0A3CA2001D0E0D6E0D2EFED7120050
:103CAC006C0E0101726F010E736F67C174F168C104
:103CBC0075F169C176F16AC177F16BC178F1720E59
:103CCC00796F010E7A6F10EC0EF000C070F101C02C
:103CDC0071F100506725E16E01506821E26EE66AD1
:0A3CEC0070C100F071C101F0120078
:103CF600C26A00017D1D006E0050C1160F0EC01273
:103D0600C08E67C100F0003600900036009000506B
:103D1600C212C280C3DFC282C2A201D0FDD7C4CF05
:103D260001F0006A00C068F101C069F1C3500012D9
:103D3600000E011200C068F101C069F1C290000EC8
:103D46000014026E0150800B036E000E031802E190
:103D5600000E021803E00101686B696B68C100F090
:063D660069C101F012002A
:103D6C0001016B6B050E6B5D0AE26B516925E16E0F
:103D7C00000E6A21E26E200EE66E6B2BF3D76B51B0
:103D8C006925E16E000E6A21E26EE66A6B076B51E3
:103D9C0069256C6F000E6A216D6F0A0E046E000EA1
:103DAC00056E67C100F068C101F05ADF08C000F071
:103DBC0009C001F0300E00266CC1E1FF6DC1E2FFBD
:103DCC0000C0E6FF0A0E046E000E056E67C100F01F
:103DDC0068C101F045DF00C067F101C068F1000E59
:103DEC00011802E1000E001801E102D06B07CFD7D9
:023DFC001200B3
:103DFE0010D0800E0101676F1AD0C00E676F17D0FA
:103E0E00940E676F14D0D40E676F11D0800E676F4B
:103E1E000ED001016751010AECE06751020AEDE094
:103E2E006751030AEDE06751040AEDE0EFD768052C
:103E3E00006E6751002600C067F100C09CF1ABEC2C
:103E4E0009F010916B6B6B516925E96E000E6A21BA
:103E5E00EA6EEE520BE06B516925E96E000E6A2197
:103E6E00EA6EEECF74F1F3DE6B2BEDD710811200FC
:103E7E0001016A6B67C1E9FF68C1EAFFEECF69F124
:103E8E006951000A0FE069C1A1F123EC01F00101B3
:103E9E006A2B6A516725E96E000E6821EA6EEECF35
:063EAE0069F1EED71200DD
:103EB4000B6A0C6A0A6A0350D8B4A4EF1FF0028E8E
:103EC4008E0E035E03BE6CEF1FF0D8B46CEF1FF0D0
:103ED400A8EF1FF0036C080E035CD8A083EF1FF05B
:103EE400036E013602C001F0026A080E035CD8A01A
:103EF40083EF1FF00136016A0350D8A4D8908DEFE8
:103F04001FF00350D8B48DEF1FF0D8900232013265
:103F1400032E87EF1FF00BBC01A09AEF1FF0D8A06F
:103F24009AEF1FF0012AD8B4022A02BEB7EF1FF09D
:103F34000AAEBDEF1FF0021E011E012AD8B4022AE8
:103F4400BDEF1FF0026A016ABDEF1FF00B800BAEDC
:103F5400C1EF1FF0026A0AAEC1EF1FF0FF0E026E3E
:103F6400016E0A360232C1EF1FF0010E0C6E38ECFE
:103F740004F0C3EF1FF0000E0C6EC3EF1FF0FF0E32
:0C3F84000C6E0150006E0250016E120025
:103F9000E80E046E030E056E67C100F068C101F003
:103FA00065DE00C007F1080E896E420EE96E000E54
:103FB000EA6E0050E926D8B0EA2AEECF8CFF640EF4
:103FC000046E000E056E67C100F068C101F04EDEA0
:103FD0000A0E046E000E056E49DE08C000F009C02E
:103FE00001F000C007F1040E896E420EE96E000E6A
:103FF000EA6E0050E926D8B0EA2AEECF8CFF8C8E0C
:104000000A0E046E000E056E67C100F068C101F073
:104010002DDE0A0E046E000E056E28DE08C000F0CC
:1040200009C001F000C007F1020E896E420EE96E70
:10403000000EEA6E0050E926D8B0EA2AEECF8CFFD7
:104040000A0E046E000E056E67C100F068C101F033
:104050000DDE08C000F009C001F000C007F1010E3C
:10406000896E420EE96E000EEA6E0050E926D8B065
:08407000EA2AEECF8CFF1200DA
:1040780069C1F6FF6AC1F7FF6BC1F8FF0900F5CF08
:1040880000F0005218E069C1F6FF6AC1F7FF6BC182
:10409800F8FF0900F5CF00F067C1E1FF68C1E2FF52
:1040A80000C0E6FF0101674B682B010E6927000E6F
:1040B8006A236B23DDD767C1E1FF68C1E2FFE66AC7
:0240C8001200E4
:1040CA000050086E0150006E016A026A036A0B6AA8
:1040DA000C6A960E036E0A6A00C001F008C000F06E
:0A40EA00086A026AD4EC0DF012001F
:1040F40067C1F6FF68C1F7FF69C1F8FF0900F5CF92
:1041040001F00150000812E267C1F6FF68C1F7FF31
:1041140069C1F8FF0900F5CFA1F123EC01F0010E0C
:0E41240001016727000E68236923E2D712000D
:1041320001016D6B6E6B000E6E5D02E10A0E6D5D2C
:104142000BE26D516B25E16E6E516C21E26E200E19
:10415200E66E6D4B6E2BEFD76D516B25E16E6E5196
:104162006C21E26EE66A010E6D5F000E6E5B6D51B0
:104172006B256F6F6E516C21706F0A0E046E000E0C
:10418200056E066E076E67C100F068C101F069C175
:1041920002F06AC103F08AEC0BF008C000F009C01B
:1041A20001F00AC002F00BC003F0300E00266FC10E
:1041B200E1FF70C1E2FF00C0E6FF0A0E046E000ECE
:1041C200056E066E076E67C100F068C101F069C135
:1041D20002F06AC103F08AEC0BF000C067F101C083
:1041E20068F102C069F103C06AF1000E046E03189F
:1041F20008E10450021805E10450011802E10050E0
:10420200000A01E105D0010E6D5F000E6E5BAFD7B3
:02421200120098
:104214000900F5CFE6FF0006FBE10106F9E1120013
:10422400460E01010C6F020E0D6FA10E0E6F010EF2
:104234000F6FFF0E196FFF0E1A6F000E1B6F000E2B
:104244001C6FFF0E156FFF0E166F000E176F000E1A
:10425400186FFF0E116FFF0E126F000E136F000E1A
:10426400146FAC8A900EAB6E948E949C9EAA03D06D
:08427400AECF00F0FBD71200F1
:10427C00FF0E0101616FFF0E626FFF0E636FFF0E89
:10428C00646FC26A00017D1D006E0050C1160F0ED6
:08429C00C012C08EC2801200A6
:1042A400939693949398939A939C939E8A968A94C4
:1042B4008A9E8A9C8A9A8A9884EC04F084EC04F09E
:1042C40084EC04F08A8A8A888A867FEC04F08A96D1
:1042D40084EC04F08A867FEC04F08A9684EC04F083
:1042E4008A867FEC04F08A9684EC04F08A988A86A5
:1042F4007FEC04F08A9684EC04F08A867FEC04F068
:104304008A968A9A8A8E8A867FEC04F08A9684EC4E
:1043140004F08A9E8A888A867FEC04F08A968A98BA
:104324008A867FEC04F08A9684EC04F08A867FEC1B
:1043340004F08A968A888A867FEC04F08A9684EC54
:1043440004F08A988A867FEC04F08A968A8E8A8C96
:104354008A8A8A888A867FEC04F08A9684EC04F040
:06436400010110811200AE
:10436A0001016A6B67C1E9FF68C1EAFFEECF69F133
:10437A006951000A0EE069C174F15EDC01016A2B21
:10438A006A516725E96E000E6821EA6EEECF69F17F
:04439A00EFD7120047
:10439E000D0E0101A16F23EC01F00A0E0101A16FB8
:0643AE0023EC01F01200F7
:1043B4008EEC25F0D38CD38AD388D382D390D3B414
:1043C40001D0FDD7799E789E816A0F01396B936A7B
:1043D400FF0E806EE00E926E100E386F896A3A6B93
:1043E400FF0E946E3C6B966AFF0E846E3B6B956A6F
:1043F4008C6AB886B06ACF0EAF6EAC8411DF030E40
:104404000B6E080E0C6E770E0D6E0D2EFED70C2E55
:10441400FCD70B2EFAD7B90E676F4A0E686F000EE1
:10442400696F66DE0D0E0101676F480E686F000E3E
:10443400696F5EDEB70E0101676F480E686F000E8C
:10444400696F56DEA30E0101676F4A0E686F000E96
:10445400696F4EDE710E0101676F490E686F000EC1
:10446400696F46DE6E0E0101676F4A0E686F000EBB
:10447400696F3EDE890E0101676F4A0E686F000E98
:10448400696F36DE470E0101676F490E686F000ED3
:10449400696F2EDE800E0101036F3E0E046F000E65
:1044A400056F066F0D0E676F4B0E686F000E696F18
:1044B4001FDE03C167F104C168F105C169F106C1DA
:1044C4006AF108C16BF109C16CF131DE08C167F111
:1044D40009C168F148DF150E676F4B0E686F000E57
:1044E400696F06DEEB0E0101676F490E686F000EFF
:1044F400696FFEDD230E0101A16F23EC01F04DDF96
:10450400660E0B6E760E0C6EC10E0D6E0D2EFED762
:104514000C2EFCD70B2EFAD7400E0101A16F23EC11
:1045240001F03BDF190E0101676F490E686F000E41
:10453400696FDEDD000E0101676F4B0E686F000EC0
:10454400696FD6DD99DEC30E0101676F490E686F8E
:10455400000E696FCDDD110E0101676F4A0E686FA1
:10456400000E696FC5DD9CDE030E0B6E080E0C6E2B
:10457400770E0D6E0D2EFED70C2EFCD70B2EFAD710
:10458400010E9C6FABEC09F00C0E9C6FABEC09F0C8
:10459400010E676F010E686F5D0E696F000E6A6F22
:1045A4002CDC020E676F010E686F4C0E696F000EF3
:1045B4006A6F23DC520E0B6E2B0E0C6E000E0D6E0A
:1045C4000D2EFED70C2EFCD70B2EFAD70000260E8C
:1045D400676F000E686F51DC010E9C6FABEC09F045
:1045E400010E676F010E686F150E696F000E6A6F1A
:1045F40004DC150E0B6E4B0E0C6EBE0E0D6E0D2EE6
:10460400FED70C2EFCD70B2EFAD7000000017E6BD0
:104614007F6B010E01019C6FABEC09F0016B026B27
:10462400000E025D02E1500E015D0AE2810E0125D9
:10463400E16E000E0221E26EE66A014B022BF0D716
:10464400810E086F000E096FC26AC16AC06AC08E0B
:10465400B20EC06E100EC26EC28000017E6B7F6B04
:10466400806B040E0101676F7BEC1EF000C00AF141
:1046740001C00BF1010E0101676F010E686F750E29
:10468400696F000E6A6FFFEC1EF07EC067F17FC099
:1046940068F1210E696F010E6A6FB6EC1EF0210EEF
:1046A400676F010E686F3FEC1FF077DE010E0101AA
:1046B400676F080E686F210E696F010E6A6FFFEC59
:1046C4001EF0210E676F010E686FEF0E696F4A0EC0
:1046D4006A6F000E6B6FCEDC0AC167F10BC168F123
:1046E4002B0E0101696F010E6A6FB6EC1EF0020E0B
:1046F400676F010E686F210E696F010E6A6FFFEC20
:104704001EF00AC100F00BC101F0DDDCF60E046EF0
:10471400280E056E1C0E066E810E076E88EC01F0E5
:1047240000C01DF101C01EF102C01FF103C020F141
:104734005AEC1FF000C065F101C066F108C167F1D1
:1047440009C168F1520E696F4A0E6A6F000E6B6FF1
:104754000AC16CF10BC16DF100C06EF101C06FF1C3
:1047640056EC1EF008C167F109C168F13FEC1FF077
:1047740065C167F166C168F109DC0B0E0B6E260E8C
:104784000C6E5D0E0D6E0D2EFED70C2EFCD70B2E6F
:10479400FAD70000000000017E4B7F2B61D7FFD7C2
:104B1C0010EE15F0690E006E010E016EA40EF66E0D
:0E4B2C00470EF76E000EF86E0AEC21F0120034
:1047A400434F4720203278313620626F6172642093
:0147B4000004
:1047B5004C6574277320676F20666F7220414443F0
:0C47C500206D656173757265200D0A009F
:0A47D1003F065B4F666D7D077F6FAA
:1047DB007769746820626F6F746C6F6164657220A7
:0147EB0000CD
:1047EC0031384634354B32322070726F746F202062
:0147FC0000BC
:0747FD00286E756C6C2900A9
:084804004D657375726520001B
:01480C000F9C
:10480D00204469726563746F7279203A433A5C5F34
:10481D004D696B726F435C5F4D657350726F6A6566
:10482D0074735F4D696B726F435C5F31384634351D
:10483D004B32325F5265616479466F725069630D18
:02484D000A005F
:10484F000000007FCDCC4C7B0AD723786F12037505
:10485F0017B75171ACC5276EBD37066B95BF56673D
:10486F0077CC2B645F700961FFE65B5D08E53C3C2C
:04487F006042221B56
:104883000000007F000020820000488500007A8835
:1048930000401C8C0050438F00247492809618961D
:1048A30020BC3E99286B6E9CF90215A0EC782DC1B3
:0448B300CAF249E21A
:1048B7002050726F6A6574203A2031384634354B80
:1048C70032325F554152545F4144435F434F473152
:1048D700365F323032305F31312E6D637070690D63
:0248E7000A00C5
:1048E9000100000008000000400000000002000074
:1048F90000100000008000000000040000002000FB
:104909000000000100000008000000400000000055
:1049190020526561647920666F72205049433138AD
:104929004634354B32322074657374204541342046
:0E49390073757220524135202121200D0A0095
:104947002055415254312076696120555342202D1C
:104957003E20434F4D3233205662726179205465B1
:0A496700726D696E616C0D0A20008C
:1049710020536F75726365203A5F31384634354B89
:1049810032325F554152545F546573745F6D737574
:0A499100746572615F2E630D0A0069
:10499B00010000000A00000064000000E8030000B2
:1049AB0010270000A086010040420F00809698005F
:0849BB0000E1F50500CA9A3B7A
:1049C30020537472617020537570706C7953656CE9
:1049D300656374206F6E2035562028666F72204CF5
:0849E30043442129200D0A00C4
:1049EB0020436865636B2064656C61792064652086
:1049FB00353030306D5320656E7472652023206521
:064A0B007420400D0A00BA
:104A1100204C434420496E69742028616C6C2077D6
:104A210069726564206F6E20506F727442200D0AA6
:014A31000084
:104A32000100000010000000000100000010000052
:104A42000000010000001000000000010000001042
:104A520020636F6E763D20253564202076616C756B
:0C4A6200653D253564206D56200D0A00CE
:104A6E002031384634354B3232205265616479201C
:0B4A7E00666F72205049430D0A2000B3
:104A8900204C434420434F473278313620737572A6
:0A4A990020504F525442200D0A0035
:104AA3002076657273696F6E203A323032305F312F
:064AB3003131350D0A004F
:104AB900204D696B726F632050726F20372E36302C
:044AC9000D0A2000B2
:104ACD003031323334353637383961626364656677
:014ADD0000D8
:104ADE003031323334353637383941424344454626
:014AEE0000C7
:104AEF005241353D414E41343D2020202020202091
:014AFF0000B6
:0D4B00002041444320696E6974200D0A00B5
:084B0D0020466F7363203D0098
:074B1500204B487A0D0A0055
:020000040030CA
:0D000100A8183CFFBD81FF0FC00FE00F40AD
:0200000400F00A
:1000000030413A45363A45383A37353A37310000CB
:100010007061756C2032392D31302D313935300019
:1000200034343A42373A45313A45393A464200008B
:100030004A6F656C6C652D3235303231393535009B
:10004000FFFFFFFFFFFFFFFFFFFFFFFFFFFFFF00BF
:10005000FFFFFFFFFFFFFFFFFFFFFFFFFFFFFF00AF
:10006000FFFFFFFFFFFFFFFFFFFFFFFFFFFFFF009F
:10007000FFFFFFFFFFFFFFFFFFFFFFFFFFFFFF008F
:10008000FFFFFFFFFFFFFFFFFFFFFFFFFFFFFF007F
:10009000FFFFFFFFFFFFFFFFFFFFFFFFFFFFFF006F
:1000A000FFFFFFFFFFFFFFFFFFFFFFFFFFFFFF005F
:1000B000FFFFFFFFFFFFFFFFFFFFFFFFFFFFFF004F
:1000C000FFFFFFFFFFFFFFFFFFFFFFFFFFFFFF003F
:1000D000FFFFFFFFFFFFFFFFFFFFFFFFFFFFFF002F
:1000E000FFFFFFFFFFFFFFFFFFFFFFFFFFFFFF001F
:1000F000FFFFFFFFFFFFFFFFFFFFFFFFFFFFFF000F
:00000001FF
